:020000040800F2
:1000000000040020E1010008E3010008E30100080A
:10001000E3010008E3010008E3010008E301000830
:10002000E3010008E3010008E3010008092F0008CC
:10003000E3010008E3010008E3010008E301000810
:10004000E3010008E3010008E3010008E301000800
:10005000E3010008E301000875310008A131000840
:10006000CD310008F931000825320008E30100080D
:10007000E3010008E3010008E3010008E3010008D0
:10008000E3010008E3010008E3010008E3010008C0
:10009000E3010008E3010008E30100085132000811
:1000A000E3010008E3010008E3010008E3010008A0
:1000B000E3010008E3010008E3010008E301000890
:1000C000E3010008E3010008E3010008E301000880
:1000D000E3010008E3010008E3010008E301000870
:1000E000B9320008E3010008E3010008E301000859
:1000F000E3010008E3010008E3010008E301000850
:10010000E3010008E3010008852F0008E30100086F
:10011000E3010008E3010008E3010008E30100082F
:10012000E3010008E3010008E3010008E30100081F
:10013000E3010008E3010008E3010008E30100080F
:10014000E3010008E3010008E3010008512600086C
:10015000E3010008E3010008E3010008E3010008EF
:10016000E3010008E3010008E3010008E3010008DF
:10017000E3010008E3010008E3010008E3010008CF
:10018000E3010008E3010008E3010008E3010008BF
:10019000E3010008E3010008E3010008E3010008AF
:1001A000E3010008E3010008E3010008E30100089F
:1001B000E3010008E3010008E3010008E30100088F
:1001C000E3010008E3010008E3010008E30100087F
:1001D000E3010008E3010008E3010008E30100086F
:1001E00002E000F000F8FEE772B6394880F30888B4
:1001F000384880F3098838484EF60851CEF200019D
:10020000086040F20000CCF200004EF63471CEF2ED
:1002100000010860BFF34F8FBFF36F8F40F2000003
:10022000C0F2F0004EF68851CEF200010860BFF334
:100230004F8FBFF36F8F4FF00000E1EE100A4EF6C4
:100240003C71CEF200010860062080F31488BFF3F1
:100250006F8F01F0C5FE02F0EDFD4FF055301F49E4
:100260001B4A91423CBF41F8040BFAE71C49194A6A
:1002700091423CBF41F8040BFAE71A491A4A1B4B5A
:100280009A423EBF51F8040B42F8040BF8E70020F5
:100290001749184A91423CBF41F8040BFAE701F0B4
:1002A000A3FE02F023FE144C144DAC4203DA54F8C2
:1002B000041B8847F9E700F03FF8114C114DAC42A0
:1002C00003DA54F8041B8847F9E701F08BBE0000FD
:1002D000000400200024002000000008000000208E
:1002E00000040020303700080024002028240020CB
:1002F0002824002068340020E0010008E001000804
:10030000E0010008E00100082DE9F04F2DED108A12
:10031000C1F80CD0C3689D46BDEC108ABDE8F08FD3
:10032000002383F311882846A047002001F0F6FA45
:1003300001F0A6FA00DFFEE770B5214C6FF07D03F7
:1003400023700423002563706FF03F061F23A57000
:10035000E57025716571A571E57125726672A372EC
:10036000E57200F0E9FC20B10F2325726672A372DA
:10037000E57201F00BFE044601F02CFE0546D8B9EB
:10038000104B9C421AD001339C4218BF054641F2E3
:10039000883404BF01250024002001F0FDFD0DB1CB
:1003A00000F0B6F800F064FD00F004FC204600F018
:1003B0000DF900F0ADF8F9E70024EDE70446EBE7AE
:1003C00028240020010007B008B500F095FBA0F13B
:1003D00020035842584108BD07B5054B02211B8830
:1003E000ADF8043001A800F0D5FB03B05DF804FBC4
:1003F000B4330008064991F8243033B100230822B1
:10040000086A81F8243000F0F7BB0120704700BF74
:10041000482400202DE9F84F234C94F82430054659
:10042000884617468BBB2E46DFF87C90002F38D0CD
:1004300094F824A0BAF1000F05D12022FF214846EC
:10044000266200F003FDCAF10805BD4228BF3D4603
:100450005FFA85FBAD0041462A4604EB8A0000F0B6
:10046000CBFC94F82430A7EB0B079B445FFA8BFB83
:10047000BBF1080F2E44A844FFB284F824B0D5D1B4
:10048000FFF7B8FF0028D1D108E0266A06EB830603
:10049000B042C9D0FFF7AEFF0028C4D10020BDE8AC
:1004A000F88F0120BDE8F88F4824002010B52023E4
:1004B00083F311881248C3680BB101F0B5FA002329
:1004C000104A0F484FF47A7101F072FA002383F357
:1004D00011880D4C236813B12368013B23606368C6
:1004E00013B16368013B6360084B1B7833B96368E1
:1004F00023B9022000F06CFC3223636010BD00BF02
:1005000034240020AD040008782900207024002045
:1005100010B5254B254953F8042F013200D110BDE9
:100520008B42F8D1224C234B22689A423AD9224B73
:100530009B6803F1006303F580439A4232D20020A6
:1005400000F052FB1D4B0220187000F031FC1C4BD8
:100550001A6C00221A64196E1A66196E596C5A6464
:10056000596E5A665A6E5A6942F080025A615A6947
:1005700022F080025A615A691A6942F000521A61E7
:100580001A6922F000521A611B6972B60D4A0E4BAD
:1005900013601B682268202181F311889D4683F334
:1005A0000888104710BD00BFFC3F00081C40000831
:1005B00004400008FF3F0008282400207024002089
:1005C0000038024008ED00E0004000082DE9F04F3F
:1005D000B04C97B020228146FF210EA8A66800F0FB
:1005E00035FCAD4A1378A346A3B9AC480121C360DA
:1005F0001170202383F31188C3680BB101F014FA42
:100600000023A74AA5484FF47A7101F0D1F90023DD
:1006100083F31188B9F1000F02D0A24BC3F8009008
:10062000A14BA04A00241C705460254627469846DA
:10063000012000F0BDFBB9F1000F00F02282994BC0
:100640001B68002B40F01D8217B0BDE8F08F022020
:10065000FFF7BAFE002840F00E82944B1B88ADF8DD
:100660002430022109A800F095FAE1E74FF47A70EE
:1006700000F042FA031E0193EFDB0220FFF7A4FE15
:1006800082460028E9D0019B581E042800F2F5811B
:10069000DFE800F0030D1013160016A8052340F83C
:1006A000343D042100F076FA5446002752E004213C
:1006B0007848F7E704217E48F4E704217D48F1E714
:1006C0001C24204600F092FA04340990042109A861
:1006D00000F060FA2C2CF4D1E6E7002DBDD0002C00
:1006E000BBD00220FFF770FE0546002800F0C7814E
:1006F000012000F079FA022088F8000000F058FB91
:100700000024E3B21846019300F07EFA824648B115
:10071000019B184600F088FA01340028F1D12C46DC
:10072000654B9BE70123022088F8003000F02EFB88
:100730005646DBF808309E4206D2304600F056FAA4
:100740000130ECD10436F4E7564B002688F80060FF
:100750005E602C4600F082FB1DB1002C18BF4FF0EC
:100760000009FFF739FE63E7002D3FF476AF002C58
:100770003FF473AF022088F8000000F019FB32202C
:1007800000F0BAF9B0F1000AC0F279811AF003055D
:1007900040F07581DBF8082006EB0A03934200F273
:1007A0006E81BAF5807F00F26A81444B0193554512
:1007B0000DDA4FF47A7000F09FF90290029A002A45
:1007C000C0F25D81019B029AEA540135EEE7C82030
:1007D000FFF7FAFD0546002800F051811F2E11D8C1
:1007E000C6F12004544528BF54460EAB26F0030042
:1007F00022463249184400F0FFFA2246FF212F48D2
:1008000000F024FB4FEAAA0A5FFA8AF22B4930462D
:10081000FFF700FE0446002881D006EB8A06054655
:1008200098E70220FFF7D0FD00283FF416AFFFF74E
:10083000E1FD00283FF411AF00229246DBF80830BA
:100840009A4259D21F2A1ED80E9B01331BD022F088
:10085000030316A90B4453F8203C09931848436836
:1008600083B3174800210DF1240E11F80E3083EAEE
:100870000A03DBB2013150F82330042983EA1A2A33
:10088000F3D10432DAE71046019200F0AFF9019A91
:100890000990E3E728240020742500203424002058
:1008A000AD0400087829002070240020B633000829
:1008B0002C24002030240020B833000874240020A9
:1008C0007825002019464FF0080E11F0010F4FEA6D
:1008D00051011FBF81F06D4181F4380181F4034162
:1008E00081F02001BEF1010EEFD140F82310013359
:1008F000B3F5807FE6D1B4E716A8042140F84CADEB
:1009000000F048F926E716A8002340F8343D64219A
:1009100000F01CF900287FF4A0AE0220FFF754FD80
:1009200000283FF49AAE099800F090F916AB43F80E
:10093000480D04211846E3E716A8002340F8343D8B
:10094000642100F003F900287FF487AE0220FFF74E
:100950003BFD00283FF481AE099800F085F916AB05
:1009600043F8440DE5E70220FFF72EFD00283FF491
:1009700074AE00F07FF916AB43F8400DD9E70220C2
:10098000FFF722FD00283FF468AE09A9142000F00B
:1009900077F9824616A8042140F83CAD00F0FAF839
:1009A000514609A8ACE7322000F0A6F8B0F1000AE1
:1009B000FFF653AE1AF0030F7FF44FAEDBF80820BA
:1009C0000AEB070393423FF648AE0220FFF7FCFC18
:1009D00000283FF442AE2AF0030ABA44BA453FF475
:1009E000B9AE384600F002F90421089008A800F0DA
:1009F000D1F80437F2E74FF47A70FFF7E5FC0028EE
:100A00003FF42BAEFFF7F6FC00283FF489AE0E9BB7
:100A100001330CD008220EA90020FFF7FBFC0028B0
:100A20003FF47EAE2022FF210EA800F00FFAFFF760
:100A3000D3FC304800F078FF06E616A8002340F803
:100A4000343D642100F082F8824600287FF405AE30
:100A50000220FFF7B9FC00283FF4FFADFFF7BCFC14
:100A600041F2883000F060FF099800F027FAD14683
:100A700000F0F4F9DCE505466CE60027EDE52546D7
:100A8000EBE5002000F038F80290029B002BFFF607
:100A9000D2AD012000F07AF9029B213B122B3FF6E8
:100AA000C7AD01A252F823F04F0600086D060008FA
:100AB000DB06000831060008310600083106000890
:100AC00069070008A70900082308000807090008AB
:100AD0003909000867090008310600087F09000885
:100AE00031060008F709000855070008310600081C
:100AF0003B0A0008A086010037B5114B1A78013275
:100B0000D2B20024012A01468DF8074011D80D48C1
:100B100003681D6A4FF47A734B4301220DF10701FC
:100B2000A847012805D1084B9DF807001C7003B0A9
:100B300030BD4FF4FA7000F0F7FE4FF0FF30F6E7EB
:100B400000240020C82900208429002038B50E4B3D
:100B50001A780132D2B2012A05460ED80B48036832
:100B60001C6A4FF47A734B4304222946A047042899
:100B700003D1074B0020187038BD4FF4FA7000F015
:100B8000D3FE4FF0FF3038BD00240020C8290020DC
:100B90008429002030B4054C2368DD69044B0A46E3
:100BA000AC460146204630BC604700BFC829002043
:100BB000A086010070B501F001F9094C094E2070C2
:100BC000002530682378834208D901F0F1F83368B2
:100BD00005440133B5F5804F3360F2D370BD00BFDB
:100BE000852900208029002001F09AB900F10060D9
:100BF00000F580400068704700F10060920000F549
:100C0000804001F025B90000054B1A68054B1B78A0
:100C10009B1A834202D9104401F0CAB800207047E1
:100C2000802900208529002038B5074D0446286812
:100C3000204401F0C5F828B928682044BDE83840B0
:100C400001F0D6B838BD00BF8029002010F00303A2
:100C500008D1B0F5007F05D800F10050A0F508409C
:100C60000068704700207047014BC058704700BFB4
:100C7000107AFF1F014B1868704700BF002004E086
:100C800070B52A4B1C68C4F30B03240C63B140F20B
:100C90001342934231D040F2194293422FD040F296
:100CA000214293422DD10323214A0C2505FB032326
:100CB0005D6893F9082042F201039C4224D0B4F508
:100CC000805F23D041F201039C4221D041F2030313
:100CD0009C421FD041F207039C4208BF3122441EB0
:100CE0000C44013D0B46A3421ED215F9016F581C5E
:100CF00096B1034600F8016CF5E70123D4E702231F
:100D0000D2E73F220B4DD6E73322E3E74122E1E76A
:100D10005A22E4E75922E2E72C2584421D7001D9CA
:100D2000981C5A70401A70BD1846FBE7002004E07A
:100D3000DC330008BC330008124B5A8842F2010130
:100D40008A4293B214D0B3F5805F13D041F201020E
:100D5000934211D041F2030293420FD041F20702B5
:100D600093420DD10423084A02EB8303D8787047DD
:100D70000023F8E70123F6E70223F4E70323F2E771
:100D800000207047002004E0C8330008022804D186
:100D9000054B4FF080429A6170470128FCD14FF417
:100DA0000012024BF7E700BF000C024000080240AF
:100DB000022804D1044B4FF480429A617047012805
:100DC000FCD12022014BF8E7000C02400008024051
:100DD000022805D1064A536983F480435361704762
:100DE0000128FCD1034A536983F02003F6E700BFD2
:100DF000000C02400008024010B50023934203D0CB
:100E0000CC5CC4540133F9E710BD000030B5441E7A
:100E100014F9010F0B4660B193F90050854201F1BE
:100E2000010106D11AB993F90020801A30BD013AA8
:100E3000EEE7002AF7D1104630BD00000246034617
:100E4000981A13F9011B0029FAD17047024403468E
:100E5000934202D003F8011BFAE77047024B1A785D
:100E6000024B1A70704700BF842900200024002024
:100E700038B50E4D0E4C284600F09EF82146284607
:100E800000F0C6F823680B485A6D936B23F40023D7
:100E9000936300F049FD0849206800F0C5F9236814
:100EA0005A6D936B43F40023936338BDC829002027
:100EB000A834000840420F00FC34000870470000CE
:100EC000026843681143016003B11847704700008E
:100ED00013B5446BD4F894341A681178042915D1E9
:100EE000217C022912D11979128901238B401342E6
:100EF0000CD101A904F14C0001F010FED4F8944487
:100F0000019B21790246206800F0DAF902B010BD99
:100F1000143001F093BD00004FF0FF33143001F0A6
:100F20008DBD00004C3001F065BE00004FF0FF3376
:100F30004C3001F05FBE0000143001F061BD0000D4
:100F40004FF0FF31143001F05BBD00004C3001F078
:100F500031BE00004FF0FF324C3001F02BBE0000DC
:100F6000D0F8942438B5136819780429054601D0BF
:100F7000012038BD017C0229FAD112795C89012057
:100F800090400440F4D105F1140001F0F3FC024656
:100F90000028EDD0D5F894544FF48073286869790F
:100FA00000F07CF9204638BD406BFFF7D9BF000048
:100FB00000207047704700007FB5124B036000238C
:100FC00043608360C360012502260F4B057404460D
:100FD0000290019300F18402294600964FF4807339
:100FE000143001F0A3FC094B0193029400964FF4D6
:100FF000807304F52372294604F14C0001F06AFD68
:1010000004B070BD2C340008A90F0008D10E0008F0
:101010000B68202282F311880A7903EB8202906127
:101020004A79093243F822008A7912B103EB82032C
:10103000986102230374C0F89414002383F3118889
:101040007047000038B5037F044613B190F8543060
:10105000ABB9201D01250221FFF732FF04F1140076
:1010600025776FF0010100F087FC84F8545004F1FB
:101070004C006FF00101BDE8384000F07DBC38BD88
:1010800010B5012104460430FFF71AFF002323772F
:1010900084F8543010BD000038B5044600251430E3
:1010A00001F05CFC04F14C00257701F02BFD201DC4
:1010B00084F854500121FFF703FF2046BDE8384073
:1010C000FFF74EBF90F8443003F06003202B19D196
:1010D00090F84520212A0AD0222A4FF000030ED092
:1010E000202A0FD1084A82630722C26304E0064B1C
:1010F00083630723C3630023036401207047836372
:10110000C363F9E70020704701240020D0F894342D
:1011100037B51A681178042904461AD1017C0229CE
:1011200017D11979128901238B40134211D100F193
:101130004C05284601F0A6FD58B101A9284601F04A
:10114000EDFCD4F89444019B21790246206800F01C
:10115000B7F803B030BD000000EB8103F7B59C6920
:1011600005460E46F4B1202383F3118805EB86076C
:10117000201D0821FFF7A4FEFB685B691B684C3447
:1011800013B1204601F0D8FC01A9204601F0C6FCAD
:10119000024648B1019B3146284600F091F80023F1
:1011A00083F3118803B0F0BDFB685A691268002A06
:1011B000F5D01B8A013B1340F1D105F14402EAE767
:1011C000093138B550F82140DCB1202383F3118870
:1011D000D4F894241368527903EB8203DB689B698B
:1011E0005D6845B104216018FFF76AFE294604F1E5
:1011F000140001F0C9FB2046FFF7B2FE002383F381
:10120000118838BD7047000000F074BF01230370DF
:1012100000234360C36183620362C362436203636A
:10122000038143817047000038B50446202383F3CF
:10123000118800254160C56005614561856100F048
:1012400069FF0223237085F3118838BD70B500EB68
:10125000810305465069DA600E46144618B1102223
:101260000021FFF7F3FDA06918B110220021FFF75C
:10127000EDFD31462846BDE8704001F015B800008C
:10128000028902F001020281428902F001024281D8
:10129000002202614261826101F09AB8F0B400EB71
:1012A00081044789E4680125A4698D403D43458157
:1012B00023600023A2606360F0BC01F0B5B80000B9
:1012C000F0B400EB81040789E468012564698D406E
:1012D0003D43058123600023A2606360F0BC01F000
:1012E0002FB9000070B50223002504460370A0F852
:1012F0004C5080F84E5080F84F5005814581C560B4
:1013000005614561856180F8345000F069FF6368CC
:101310001B6823B129462046BDE87040184770BDC0
:10132000436802781B6880F85020052202700BB1D8
:101330000421184770470000436890F850201B684C
:1013400002700BB1052118477047000090F8343047
:1013500070B5044613B1002380F8343004F1440220
:10136000204601F057F863689B6863BB94F84450CB
:1013700015F0600615D194F8453005F07F0545EA73
:10138000032540F202339D4200F00E815BD8022D0E
:1013900000F0DC803FD8002D00F08780012D00F0A8
:1013A000CF800021204601F08DFA0021204601F077
:1013B0007FFA63681B6813B106212046984706230D
:1013C00084F8343070BD204698470028CED094F879
:1013D0004B2094F84A3043EA0223E26B934238BF31
:1013E000E36394F94430E56B002B4FF0200380F267
:1013F000FD80002D00F0EC80092284F8342083F376
:1014000011880021E36BA26B2046FFF759FF0023F0
:1014100083F3118870BDB5F5817F00F0B180B5F51B
:10142000407F49D0B5F5807FBBD194F84630012B81
:10143000B7D1B4F84C3023F00203A4F84C30A663C3
:10144000E6632664C3E740F201639D421ED8B5F50A
:10145000C06F3BD2B5F5A06FA3D1B4F84430B3F55B
:10146000A06F0ED194F8463084F84E30204600F03C
:101470000FFF63681B6813B10121204698470323BF
:1014800023700023A363E3632364A0E7B5F5106F23
:1014900032D040F602439D4252D0B5F5006F80D164
:1014A00004F14F03A363012324E004F14C03A3637D
:1014B0000223E36325648AE794F84630012B7FF426
:1014C00070AFB4F84C3043F00203B6E794F849200B
:1014D000616894F848304D6894F8471043EA022355
:1014E000204694F84620A84700283FF45AAF4368A6
:1014F000A3630368E363A4E72378042B10D12023BC
:1015000083F311882046FFF7BBFE86F311886368DA
:1015100084F84F601B68032121700BB12046984767
:1015200094F84630002BACD084F84F30042323705D
:1015300063681B68002BA4D0022120469847A0E7CF
:10154000374BA3630223E36300239DE794F848101D
:1015500011F0800F204601F00F010ED000F04CFF7B
:10156000012806D002287FF41CAF2E4BA363E06352
:1015700067E72D4BA363E56363E700F02FFFEFE719
:1015800094F84630002B7FF40CAF94F8483013F0F9
:101590000F013FF476AF1A06204602D501F0A6F9F6
:1015A0006FE701F099F96CE794F84630002B7FF46F
:1015B000F8AE94F8483013F00F013FF462AF1B0609
:1015C000204602D501F07EF95BE701F071F958E79A
:1015D000142284F8342083F311882B462A462946A6
:1015E0002046FFF75BFE85F3118870BD5DB11522C3
:1015F00084F8342083F311880021E36BA26B20462A
:10160000FFF74CFE03E70B2284F8342083F31188A4
:101610002B462A4629462046FFF752FEE3E700BF45
:101620005C340008543400085834000838B590F889
:1016300034300446152B29D8DFE803F03E2828284B
:1016400028283E28280B293928282828282828280F
:101650003E3E90F84B1090F84A20C36B42EA0122BC
:101660009A4214D9C268128AB3FBF2F502FB15350F
:101670006DB9202383F311882B462A462946FFF7AC
:101680001FFE85F311880A2384F8343038BD1423F3
:1016900084F83430202383F3118800231A46194636
:1016A0002046FFF7FBFD002383F3118838BD036C50
:1016B00003B198470023E7E7002101F003F9002177
:1016C000204601F0F5F863681B6813B10621204637
:1016D00098470623D8E7000090F83420152A38B53B
:1016E000044622D80123934040F6416213421DD1A3
:1016F00013F480150FD19B0217D50B2380F83430DB
:10170000202383F311882B462A462946FFF7D8FD6C
:1017100085F3118838BDC3689B695B682BB9036C7E
:1017200003B19847002384F8343038BD002101F01C
:10173000C9F80021204601F0BBF863681B6813B1AB
:101740000621204698470623EDE70000024B0022C1
:101750001B605B609A607047882900200023037437
:101760008268054B1B6899689142FBD25A680360F6
:1017700042601060586070478829002008B5202317
:1017800083F31188037C032B05D0042B0DD02BB9D8
:1017900083F3118808BD436900221A604FF0FF33BC
:1017A0004361FFF7DBFF0023F2E790E80C001A60CB
:1017B00002685360F2E70000002303748268054B5F
:1017C0001B6899689142FBD85A68036042601060B8
:1017D0005860704788290020054B196908741868FB
:1017E00002681A605360186101230374FEF78CBD10
:1017F0008829002030B54B1C87B005460A4C10D014
:1018000023690A4A01A800F0D3F82846FFF7E4FF4D
:10181000049B13B101A800F007F92369586907B0C8
:1018200030BDFFF7D9FFF8E7882900207D170008B1
:1018300038B50C4D41612B6981689A689142044624
:1018400003D8BDE83840FFF789BF1846FFF786FF89
:1018500001232C61014623742046BDE83840FEF781
:1018600053BD00BF88290020044B1A681B6990688B
:101870009B68984294BF002001207047882900206F
:1018800010B5084C236820691A6822605460012250
:1018900023611A74FFF790FF01462069BDE81040EC
:1018A000FEF732BD882900208260022202740022E5
:1018B000427470478368A3F17C0243F80C2C0269E0
:1018C00043F83C2C426943F8382C074A43F81C2C57
:1018D000C26843F8102C022203F8082C002203F8F7
:1018E000072CA3F1180070472103000810B520232E
:1018F00083F31188FFF7DEFF00210446FFF798FF0E
:10190000002383F31188204610BD0000024B1B69A1
:1019100058610F20FFF760BF88290020202383F340
:101920001188FFF7F3BF000008B50146202383F3B9
:1019300011880820FFF75EFF002383F3118808BD9C
:1019400049B1064B42681B6918605A6013604360D6
:101950000420FFF74FBF4FF0FF3070478829002069
:101960000368984206D01A680260506059611846B0
:10197000FFF7F4BE7047000038B504460D462068F6
:10198000844200D138BD036823605C604561FFF785
:10199000E5FEF4E7054B03F114025A619A614FF03A
:1019A000FF32DA6100221A62704700BF88290020E6
:1019B000F8B503611A4BC2605C6A1A4B1A460229D9
:1019C00052F8145F38BF0221954206461F460AD1DD
:1019D000586198611C620560456081600819BDE826
:1019E000F84001F071B9186AAB68241A0C1902D3D7
:1019F000E41A2D6804E09C4202D2204401F074F9FC
:101A0000AB689C42F4D86B68736035601E606E6092
:101A1000B460A9684FF0FF33091BA960FB61F8BDF2
:101A2000000C00408829002010B41A4C234653F8BB
:101A3000141F814210D0416802680A600268516038
:101A40009A424FF00001C16003D0936881680B4453
:101A500093605DF8044B70470A68626100209A4207
:101A60005360C86003D15DF8044B01F037B9936847
:101A7000886803449360084A206A526A121A9342A3
:101A8000E7D9991A012998BF931C18445DF8044BB3
:101A900001F02AB988290020000C0040002070477E
:101AA000FEE70000704700004FF0FF307047000075
:101AB000022906D0032906D00129064818BF0020B4
:101AC000704705487047032A9ABF044800EBC200DC
:101AD00000207047583500080C3500080824002005
:101AE00070B5044608460D46FFF7A8F9C6B2204671
:101AF000013403780BB9184670BD32462946FFF70A
:101B000085F90028F3D1012070BD00002DE9F04FC8
:101B100081469BB008460D461646FFF78FF93D49B2
:101B2000C4B22846FFF7DCFF08B10434E4B23A49F6
:101B30002846FFF7D5FF08B11034E4B2632C01AF9B
:101B40000CD8DFF8E0A0DFF8E0B03C4695F8008064
:101B5000B8F1000F1CD184F8008003E02946384614
:101B600001F020FC3846FFF769F9C0B2431C5B0066
:101B700089E8480033700323737000230236194646
:101B8000DAB2904206F102063DD81BB0BDE8F08FF4
:101B9000B8F1250F32D107221E492846FFF736F942
:101BA00070B9DBF800202260DBF804206260BBF82B
:101BB000082022819BF80A20A27207350B34C5E762
:101BC000082215492846FFF721F9B8B91348A21C85
:101BD00010F8011F124B4FEA111E01F00F011EF801
:101BE0000AE011F80A1002F802EC984202F8011C0F
:101BF00002F10202ECD118340835A7E784F800801E
:101C000001350134A2E7FA5C06F8022C06F8011C43
:101C10000133B5E7B0340008B83400080F7AFF1F6D
:101C20001B7AFF1FCD340008C134000808B52023FB
:101C300083F311880348FFF769FA002383F31188BF
:101C400008BD00BFC829002010B50446052916D8D4
:101C5000DFE801F016150316161D202383F3118803
:101C60000E4A0121FFF7F2FA20460D4A0221FFF742
:101C7000EDFA0C48FFF710FA002383F3118810BD2A
:101C8000202383F311880748FFF7DCF9F4E72023CA
:101C900083F311880348FFF7F3F9EDE76034000898
:101CA00084340008C829002038B50C4D0C4C0D496F
:101CB0002A4604F10800FFF729FF05F1CA0204F1E2
:101CC00010000949FFF722FF05F5CA7204F1180058
:101CD0000649BDE83840FFF719BF00BF902E00202D
:101CE00008240020E0340008F1340008B83400086B
:101CF000BFF34F8F024AD368DB03FCD4704700BFA9
:101D0000003C024008B5094B1B7873B9FFF7F0FFA0
:101D1000074B1A69002ABFBF064A5A6002F188328F
:101D20005A601A6822F480621A6008BDEE30002002
:101D3000003C02402301674508B50B4B1B7893B963
:101D4000FFF7D6FF094B1A6942F000421A611A6880
:101D500042F480521A601A6822F480521A601A689B
:101D600042F480621A6008BDEE300020003C024060
:101D7000172870B513D80B4A0B4C137863B90B4E68
:101D80004FF0006144F8231056F823500133182B0C
:101D90002944F7D10123137054F8200070BD0020AE
:101DA00070BD00BF50310020F030002078350008B1
:101DB000014B53F820007047783500081820704711
:101DC000172810B5044601D9002010BDFFF7D0FF39
:101DD000064B53F824301844C21A0BB9012010BD29
:101DE00012680132F0D1043BF6E700BF78350008F5
:101DF000172810B5044626D8FFF77AFFFFF782FFB1
:101E00001249F323CB60FFF773FF0C23B0FBF3F20F
:101E100003FB1200D30143EAC003DBB243F40073B7
:101E200043F002030B610B6943F480330B61FFF74E
:101E30005FFF2046FFF79CFFFFF77EFF2046BDE8CF
:101E40001040FFF7BDBF002010BD00BF003C0240A6
:101E50002DE9F84312F00103154643D10244B2F1D3
:101E6000026F3FD22C4B1B6813F001033AD02B4C6E
:101E7000FFF748FFF323E360FFF73AFF40F2012743
:101E8000032D16D8254C0F46401A40F20118EB1BC3
:101E90000B44012B00EB0706236926D823F001032E
:101EA0002361FFF749FF0120BDE8F883043D0430BA
:101EB000E6E78307E6D1236923F4407323612369AE
:101EC0003B43236151F8046B0660BFF34F8FFFF76C
:101ED0000FFF03689E42E9D0236923F001032361C9
:101EE000FFF72AFF0020BDE8F88323F44073236145
:101EF000236943EA08032361B94637F8023B33807C
:101F0000BFF34F8FFFF7F4FE3688B9F80030B6B252
:101F1000B342BCD0E0E700BF00380240003C0240C2
:101F2000084908B50B7828B153B9FFF7EBFE012338
:101F30000B7008BD23B1BDE808400870FFF7FCBE78
:101F400008BD00BFEE300020014B53F82000704761
:101F5000502800400A4B1A6F120407D41A6F42F43B
:101F600000721A671A6F42F400421A67054A136832
:101F700043F48073136000B2034B43F820107047A2
:101F8000003802400070004050280040014B1868A3
:101F9000704700BF5028004001460020FFF7DABF1D
:101FA00038B5094B1B689B000CD5084B084D012226
:101FB0001A700024E0B2FFF7C7FF45F8240001348F
:101FC000082CF7D138BD00BF7438024074310020AE
:101FD00054310020014B1878704700BF7431002045
:101FE00070470000FEE70000084A094B09498B4290
:101FF00004D3094A0021934205D3704752F8040FD5
:1020000043F8040BF3E743F8041BF4E754370008E4
:10201000683400206834002068340020836D30B5B7
:1020200000229D68446D11464FF0FF3004EB4213CF
:1020300001329542C3F80019C3F81019C3F8080912
:10204000C3F8001BC3F8101BC3F8080BEED24FF007
:102050000113C4F81C3830BD890141F02001016131
:1020600003699B06FCD4122000F0CABE204B03EB90
:1020700080022DE9F047D2F80CE05D6DDEF8142007
:10208000461CD2F800C005EB063605EB4018516837
:1020900061450BD3D5F83428012303FA00F022EA76
:1020A0000000C5F834081846BDE8F087BEF81040B7
:1020B000ACEB0103A34228BF2346D8F81849A4B2C9
:1020C000B3EB840F10D894681F46A4F1040959F8A3
:1020D00004AFC6F800A0042F01D9043FF7E71C4461
:1020E0000B4494605360D2E70020BDE8F08700BF46
:1020F0007831002010B5054C2046FFF787F84FF0E7
:10210000A0436365024BA36510BD00BF783100207A
:10211000FC3500080378012B70B5054650D12A4BD9
:10212000446D98421BD1294B5A6B42F080025A638E
:102130005A6D42F080025A655A6D5A6942F0800227
:102140005A615A6922F080025A610E2143205B696C
:1021500000F0D6FB1E4BE3601E4BC4F80038002392
:10216000C4F8003EC02323606E6D4FF45023A36378
:102170003369002BFCDA012333610C2000F040FEB0
:102180003369DB07FCD4122000F03AFE3369002BE0
:10219000FCDA0026A6602846FFF740FF6B68C4F80B
:1021A0001068DB68C4F81468C4F81C684BB90A4BA3
:1021B000A3614FF0FF336361A36843F00103A360A1
:1021C00070BD064BF4E700BF7831002000380240B4
:1021D0004014004003002002003C30C0083C30C0E6
:1021E000F8B5446D054600212046FFF735FFA96D7F
:1021F00000234FF001128F68C4F834384FF00066A6
:10220000C4F81C284FF0FF3004EB431201339F4207
:10221000C2F80069C2F8006BC2F80809C2F8080BDE
:10222000F2D20B686A6DEB65636210231361166965
:1022300016F01006FBD1122000F0E2FDD4F80038B1
:1022400023F4FE63C4F80038A36943F4402343F049
:102250001003A3610923C4F81038C4F814380A4BDA
:10226000EB604FF0C043C4F8103B084BC4F8003B90
:10227000C4F81069C4F80039EB6D03F1100243F49F
:102280008013EA65A362F8BDD835000840800010CD
:10229000426D90F84E10D2F8003823F4FE6343EA02
:1022A0000113C2F8003870472DE9F0410EB200EB7F
:1022B00086080D46D8F80C100F6807F00303022BB0
:1022C00050D0032B50D03D4A3D4F012B18BF17462D
:1022D000446D4FEA451E04EB0E030022C3F8102B99
:1022E0008A6905F1100C002A40D04A8A05F158038A
:1022F0005B013A43E2500123D4F81C2803FA0CF3A3
:102300001343A6444A69C4F81C380023CEF8103998
:1023100005F13F03002A39D00A8A898B92080129E6
:1023200088BF4A43C16D04EB8303561841EA024259
:10233000C66529465A602046FFF78EFED8F80C3055
:102340001B8A43EA85531F4305F148035B01E750AD
:102350000123D4F81C2803FA05F51543C4F81C58CA
:10236000BDE8F081174FB3E7174FB1E704EB461311
:10237000D3F8002B22F40042C3F8002BD4F81C2819
:10238000012303FA0CF322EA0303BAE704EB830305
:102390000E4A5A6004EB461629462046FFF75CFEBB
:1023A000D6F8003923F40043C6F80039D4F81C38B5
:1023B000012202FA05F523EA0505CFE700800010A7
:1023C000008004100080081000800C10000400023F
:1023D000826D1268C265FFF721BE00005831436D5F
:1023E00049015B5813F4004004D013F4001F14BFDC
:1023F00001200220704700004831436D49015B58BD
:1024000013F4004004D013F4001F14BF0120022075
:102410007047000000EB8101CB68196A0B681360FC
:102420004B6853607047000000EB810330B5DD68F6
:10243000AA691368D36019B9402B84BF4023136085
:102440006B8A1468426D1C44013CB4FBF3F4634393
:10245000033323F0030302EB411043EAC44343F088
:10246000C043C0F8103B2B6803F00303012B09B2F3
:102470000ED1D2F8083802EB411013F4807FD0F867
:10248000003B14BF43F0805343F00053C0F8003BBF
:1024900002EB4112D2F8003B43F00443C2F8003B88
:1024A00030BD00002DE9F041244D6E6D06EB401368
:1024B0000446D3F8087BC3F8087B38070AD5D6F85A
:1024C0001438190706D505EB84032146DB68284636
:1024D0005B689847FA072FD5D6F81438DB072BD559
:1024E00005EB8403D968CCB98B69488A5E68B6FB72
:1024F000F0F200FB12628AB91868DA6890420DD2D5
:10250000121A83E81400202383F311880B48214614
:10251000FFF78AFF84F31188BDE8F081012303FAF5
:1025200004F26B8923EA02036B81CB6823B1214655
:102530000248BDE8F0411847BDE8F081783100203D
:1025400000EB810370B5DD68436D6C692668E66059
:102550004A0156BB1A444FF40020C2F810092A68F9
:1025600002F00302012A0AB20ED1D3F8080803EBE5
:10257000421410F4807FD4F8000914BF40F080505A
:1025800040F00050C4F8000903EB4212D2F80009F1
:1025900040F00440C2F80009D3F83408012202FADE
:1025A00001F10143C3F8341870BD19B9402E84BF3E
:1025B0004020206020682E8A841940F00050013CA1
:1025C0001A44B4FBF6F440EAC440C6E7F8B5044642
:1025D0001E48456D05EB4413D3F80869C3F8086934
:1025E000F10717D5D5F81038DA0713D500EB8403B7
:1025F000D9684B691F68DA68974218D2D21B002746
:102600001A605F60202383F311882146FFF798FF4B
:1026100087F31188330617D5D5F834280123A34052
:10262000134211D02046BDE8F840FFF71FBD01233B
:1026300003FA04F2038923EA020303818B68002B67
:10264000E8D021469847E5E7F8BD00BF7831002083
:1026500096482DE9F84F456D6E69AB691E4016F43A
:10266000805F6E61044605D0FEF73CFEBDE8F84F82
:1026700000F05ABC002E12DAD5F8003E8B489B07BA
:102680001EBFD5F8003E23F00303C5F8003ED5F881
:10269000043823F00103C5F80438FEF74DFE370572
:1026A00002D58248FEF73CFEB0040CD5D5F80838B8
:1026B00013F0060FEB6823F470530CBF43F4105370
:1026C00043F4A053EB60310704D56368DB680BB1BA
:1026D00076489847F2025AD4B3020CD5D4F8548005
:1026E000DFF8C8A100274FF00109A36D9B68F9B27C
:1026F0008B4280F08780F70619D5616D0A6AC2F3B4
:102700000A1702F00F0302F4F012B2F5802F00F066
:10271000A180B2F5402F0AD104EB830301F580516B
:10272000DB68186A00231A469F4240F08780300316
:10273000D5F8184813D5E10302D50020FFF7B2FE03
:10274000A20302D50120FFF7ADFE630302D50220EC
:10275000FFF7A8FE270302D50320FFF7A3FE7503AA
:1027600084D5E00702D50020FFF730FFA10702D58E
:102770000120FFF72BFF620702D50220FFF726FF9B
:1027800023077FF573AF0320FFF720FF6EE7D4F830
:102790005480DFF818A100274FF00109A36D9B6852
:1027A0005FFA87FB5B4597D308EB4B13D3F80029FF
:1027B00002F44022B2F5802F22D1D3F80029002A5A
:1027C0001EDAD3F8002942F09042C3F80029D3F86A
:1027D0000029002AFBDB5946606DFFF73DFC22898A
:1027E00009FA0BF322EA0303238104EB8B03DB6872
:1027F0009B6813B15946504698475846FFF736FC38
:102800000137CBE708EB4112D2F8003B03F4402339
:10281000B3F5802F10D1D2F8003B002B0CDA62897F
:1028200009FA01F322EA0303638104EB8103DB6805
:10283000DB680BB150469847013756E79C0708BF45
:102840000A68072B98BF027003F101039CBF120AAC
:10285000013069E7023304EB830201F580515268CD
:1028600090690268D0F808C04068A2EB000E002210
:10287000104697420AD104EB830463689B699A6807
:102880003A449A605A6817445F6050E712F0030FA9
:1028900008BF0868964588BF8CF8000002F1010265
:1028A00084BF000A0CF1010CE3E700BF783100207F
:1028B000436D03EB4111D1F8003B43F40013C1F821
:1028C000003B7047436D03EB4111D1F8003943F4ED
:1028D0000013C1F800397047436D03EB4111D1F883
:1028E000003B23F40013C1F8003B7047436D03EB3A
:1028F0004111D1F8003923F40013C1F800397047B1
:1029000000F1604300F01F02400903F56143090133
:102910008000C9B200F1604083F8001300F5614007
:1029200001239340C0F880310360704730B5039CA9
:102930000172043304FB0325C361049B036300217C
:10294000059B00604060C160426102618561046274
:1029500042628162C162436330BD00000022416A6D
:1029600041610161C2608262C2626FF00101FFF7E2
:1029700003B8000003694269934203D1C2680AB1F7
:1029800000207047181D704703691960C268013242
:10299000C260C269134482690361934224BF436ADF
:1029A00003610021FEF7DCBF38B504460D46E3683D
:1029B0003BB16269131D1268A3621344E3620020F5
:1029C00038BD237A33B929462046FEF7B9FF0028DF
:1029D000EDDA38BD6FF00100FBE70000C368C269A3
:1029E000013BC3604369134482694361934224BF3E
:1029F000436A436100238362036B03B11847704746
:102A000070B52023044683F31188866A3EB9FFF728
:102A1000CBFF054618B186F31188284670BDA36A1E
:102A2000E26A13F8015BA362934202D32046FFF7E8
:102A3000D5FF002383F31188EFE700002DE9F84F5D
:102A400004460E4690469946202787F311880025B4
:102A5000AA46D4F828B0BBF1000F09D14946204658
:102A6000FFF7A2FF20B18BF311882846BDE8F88F4D
:102A7000A16AE36AA8EB050B5B1A9B4528BF9B463E
:102A8000BBF1400F1BD9334601F1400251F8040B52
:102A900043F8040B9142F9D1A36A40334036A36254
:102AA0004035A26AE36A9A4202D32046FFF796FFB6
:102AB0008AF311884545D8D287F31188C9E7304693
:102AC0005A46FEF799F9A36A5B445E44A3625D44EB
:102AD000E7E7000010B5029C0172043303FB0421F8
:102AE000C36100238362C362039B0363049B006092
:102AF0004060C4604261026181610462426243637A
:102B000010BD0000026AC260426A42610261002296
:102B10008262C2626FF00101FEF72EBF4369026953
:102B20009A4203D1C2680AB100207047184650F893
:102B3000043B0B6070470000C368C2690133C36087
:102B40004369134482694361934224BF436A4361EA
:102B50000021FEF705BF000038B504460D46E368C6
:102B60003BB123691A1DA262E2691344E3620020AB
:102B700038BD237A33B929462046FEF7E1FE002806
:102B8000EDDA38BD6FF00100FBE700000369196062
:102B9000C268013AC260C269134482690361934208
:102BA00024BF436A036100238362036B03B11847A8
:102BB0007047000070B5202304460E4683F3118849
:102BC000856A35B91146FFF7C7FF10B185F3118843
:102BD00070BDA36A1E70A36AE26A01339342A362C6
:102BE00004D3E16920460439FFF7D0FF002080F3C9
:102BF000118870BD2DE9F84F04460D4691469A465E
:102C00004FF0200888F311880026B346A76A4FB911
:102C100051462046FFF7A0FF20B187F311883046C8
:102C2000BDE8F88FA06AE76AA9EB06033F1A9F4246
:102C300028BF1F46402F1BD905F1400355F8042B30
:102C400040F8042B9D42F9D1A36A4033A362403679
:102C5000A26AE36A9A4204D3E16920460439FFF785
:102C600095FF8BF311884E45D9D288F31188CDE7B3
:102C700029463A46FEF7C0F8A36A3B443D44A362A6
:102C80003E44E5E7026943699A4203D1C3681BB930
:102C9000184670470023FBE7836A002BF8D0043BFB
:102CA0009B1AF5D01360C368013BC360C3691A4423
:102CB000836902619A4224BF436A036100238362ED
:102CC0000123E5E700F072B9034B002258631A6153
:102CD0000222DA60704700BF000C0040014B002266
:102CE000DA607047000C0040014B5863704700BF2A
:102CF000000C0040FEE7000010B5174CFEF726FD63
:102D0000FEF748FE802215492046FEF7CDFD01233F
:102D100044F8180C0374124B124AD96821F4E0618C
:102D20000904090C0A431049DA60CA6842F080724B
:102D3000CA600E490A6842F001020A601022DA777E
:102D4000202283F82220002383F3118862B60848EA
:102D5000BDE81040FEF7CABDB029002008360008C3
:102D600000ED00E00003FA05F0ED00E0001000E0E7
:102D7000103600082DE9F84F1F4CDFF88090656988
:102D800004F114074FF00008D9F82430266AAA6825
:102D90009E1B96421DD34FF0200AAA68236AD5F8DD
:102DA0000CB0134423622B68BB425F60A6EB0206A3
:102DB0006361C5F80C8001D1FFF790FF88F311889B
:102DC0002869D8478AF311886569AB689E42E4D2C6
:102DD000DAE76269BA420CD0916823628E1B966072
:102DE000A86802282CBF1818981CBDE8F84FFFF7F8
:102DF0007BBFBDE8F88F00BF88290020000C004091
:102E0000034B59685A68521A9042FBD8704700BF6A
:102E1000001000E04B6843608B688360CB68C36040
:102E20000B6943614B6903628B6943620B68036002
:102E30007047000008B5224B22481A6940F2FF1182
:102E40000A431A611A6922F4FF7222F001021A6120
:102E50001A691A6B0A431A631A6D0A431A651A4AE9
:102E60001B6D1146FFF7D6FF184802F11C01FFF752
:102E7000D1FF174802F13801FFF7CCFF154802F1E6
:102E80005401FFF7C7FF144802F17001FFF7C2FFBA
:102E9000124802F18C01FFF7BDFF114802F1A801B1
:102EA000FFF7B8FF0F4802F1C401FFF7B3FF0E4868
:102EB00002F1E001FFF7AEFFBDE8084000F0E2B824
:102EC0000038024000000240303600080004024092
:102ED00000080240000C02400010024000140240B2
:102EE00000180240001C02400020024008B500F01B
:102EF0003DFAFFF701FFFFF753F8BDE80840FEF782
:102F0000D3BE000070470000064A536823F0010357
:102F10005360EFF30983683383F30988002383F355
:102F20001188704730EF00E010B5202383F311883B
:102F3000104B5B6813F4006318D0F1EE103AEFF316
:102F400009844FF0807344F84C3C0B4BDB6844F829
:102F5000083CA4F1680383F30988FEF785FC18B1E7
:102F6000064B44F8503C10BD054BFAE783F311883B
:102F700010BD00BF00ED00E030EF00E031030008BD
:102F800034030008084B1A69920710B508D50024CD
:102F90001C61202383F31188FFF7ECFE84F3118872
:102FA000BDE81040FFF7C0BF000C0040104B1A6C8A
:102FB00042F008021A641A6E42F008021A660D4ABC
:102FC0001B6E936843F0080393600B4B53229A6285
:102FD0004FF0FF32DA6200229A615A63DA605A6077
:102FE00001225A6108211A603220FFF789BC00BF14
:102FF00000380240002004E0000C00401F4B1A691A
:103000006FEAC2526FEAD2521A611A69C2F3080219
:103010001A614FF0FF301A695A69586100215A69E4
:1030200059615A691A6A62F080521A621A6A02F089
:1030300080521A621A6A5A6A58625A6A59625A6AFD
:103040001A6C42F080521A641A6E42F080521A666C
:103050001A6E0B4A106840F480701060186F00F40C
:103060004070B0F5007F1EBF4FF4803018671967BD
:10307000536823F40073536000F058B900380240DD
:1030800000700040324B4FF080521A64314A4FF4C6
:10309000404111601A6842F001021A601A689207F2
:1030A000FCD59A6822F003029A60294B19469A6867
:1030B00012F00C02FBD1186800F0F90018609A6059
:1030C0001A6842F480321A600B689B03FCD54B6F80
:1030D00043F001034B671E4B5A6F9007FCD51E4A05
:1030E0005A601A6842F080721A601A4A536859048A
:1030F000FCD5174B1A689201FCD5184A9A60032236
:10310000C3F88C20164B1A68164B9A42164B1BD1EB
:10311000164A1168164A914216D140F205121A60F9
:103120000B4B9A6842F002029A609A6802F00C0215
:10313000082AFAD15A6C42F480425A645A6E42F418
:1031400080425A665B6E704740F20572E7E700BF47
:10315000003802400070004018544007009488383E
:10316000002004E011640020003C024000ED00E07B
:1031700041C20F41084A08B5536911680B4003F07A
:103180000103536123B1054A13680BB15068984796
:10319000BDE80840FFF7C8BE003C0140E83300200E
:1031A000084A08B5536911680B4003F002035361E4
:1031B00023B1054A93680BB1D0689847BDE8084031
:1031C000FFF7B2BE003C0140E8330020084A08B5D2
:1031D000536911680B4003F00403536123B1054A9E
:1031E00013690BB150699847BDE80840FFF79CBED2
:1031F000003C0140E8330020084A08B553691168D3
:103200000B4003F00803536123B1054A93690BB1E6
:10321000D0699847BDE80840FFF786BE003C0140F2
:10322000E8330020084A08B5536911680B4003F0E1
:103230001003536123B1054A136A0BB1506A9847D2
:10324000BDE80840FFF770BE003C0140E8330020B5
:10325000174B10B55C691A68144004F478725A610F
:10326000A30604D5134A936A0BB1D06A9847600647
:1032700004D5104A136B0BB1506B9847210604D547
:103280000C4A936B0BB1D06B9847E20504D5094A01
:10329000136C0BB1506C9847A30504D5054A936C89
:1032A0000BB1D06C9847BDE81040FFF73DBE00BFA2
:1032B000003C0140E83300201A4B10B55C691A68E5
:1032C000144004F47C425A61620504D5164A136D19
:1032D0000BB1506D9847230504D5134A936D0BB17C
:1032E000D06D9847E00404D50F4A136E0BB1506EB1
:1032F0009847A10404D50C4A936E0BB1D06E984741
:10330000620404D5084A136F0BB1506F9847230429
:1033100004D5054A936F0BB1D06F9847BDE81040B4
:10332000FFF702BE003C0140E8330020062108B54B
:103330000846FFF7E5FA06210720FFF7E1FA062124
:103340000820FFF7DDFA06210920FFF7D9FA062148
:103350000A20FFF7D5FA06211720FFF7D1FA062138
:103360002820BDE80840FFF7CBBA000008B5FFF7FA
:1033700045FE00F00BF8FDF747FFFDF71BFEFFF7DA
:10338000C1FDBDE80840FFF79DBC000000230449D3
:103390001A465A50C8180833802B4260F9D170473A
:1033A000E8330020034611F8012B03F8012B002A13
:1033B000F9D17047121012131211000053544D33FB
:1033C00032463F3F3F000000012033000010410122
:1033D00001105A01031059010710310100000000CB
:1033E000BC3300083F000000130400000C34000848
:1033F0003F00000019040000163400083F000000E0
:1034000021040000203400083F00000053544D33D5
:1034100032463430780053544D33324634327800DB
:1034200053544D33324634343658580000000000AF
:103430002D0F0008190F0008550F0008410F000854
:103440004D0F0008390F0008250F0008110F000864
:10345000B10F0008000000000100000000000000A3
:10346000020000000000000059110008C11100080E
:1034700040004000602E0020702E0020020000005E
:10348000000000000300000000000000051200081A
:103490000000000010000000802E0020000000004E
:1034A000010000000000000078310020010102004E
:1034B00025424F41524425002553455249414C2550
:1034C000005652427261696E2D76353400303132C9
:1034D00033343536373839414243444546000000DD
:1034E0004C61736572204E617669676174696F6EB5
:1034F0000025424F415244252D424C00491C0008F2
:10350000B11A0008C51000082D1C00084300000077
:103510001435000809024300020100C0320904000A
:103520000001020201000524001001052401000130
:10353000042402020524060001070582030800FF97
:1035400009040100020A0000000705010240000012
:1035500007058102400000001200000060350008ED
:103560001201100102000040AC27541100020102B8
:1035700003010000040309040040000000400000B3
:1035800000400000004000000000010000000200B8
:103590000000020000000200000002000000020023
:1035A0000000020000000200004000000040000097
:1035B0000040000000400000000001000000020088
:1035C00000000200000002000000020000000200F3
:1035D0000000020000000200000000004D1300087F
:1035E0002D160008D916000840004000D8310020F0
:1035F000D831002001000000E831002080000000E8
:1036000040010000030000006D61696E00000000D1
:1036100028360008F0310020E833002001000000C7
:10362000F52C00080000000069646C6500000000D3
:103630000000802A00000000AAAAAAAA0000000038
:10364000FFFF00000000000000A00A0000000000D2
:1036500000000000AAAAAAAA00000000FFFF0000C4
:103660000000000000000000000400000000000056
:10367000AAAAAAAA00000000FFFF000000000000A4
:10368000000000000000001000000000AAAAAAAA82
:1036900000000000FFFF000000000000000000002C
:1036A0000000000000000000AAAAAAAA0000000072
:1036B000FFFF00000000000000000000000000000C
:1036C00000000000AAAAAAAA00000000FFFF000054
:1036D00000000000000000000000000000000000EA
:1036E000AAAAAAAA00000000FFFF00000000000034
:1036F0000000000000000000000000000A000000C0
:1037000000000000030000000000000000000000B6
:1037100000000000000000000000000000000000A9
:103720000000000000000000000000000000000099
:10373000FF00960000000008040000007435000837
:103740000000000000000000000000000000000079
:08375000000000000000000071
:00000001FF
